:040000008A152E2C03
:08000800FF00030EF0000A0ED8
:0C001000F100040EF2008A150A12322CD6
:10002000AC08031D14280800023000000000FF3E49
:10003000031D152800000000AC0B14280800A508BB
:10004000031D23280800CC30000000000000000041
:10005000FF3E031D24280000000000000000A50B47
:1000600023280800831203171F0A9F00193A031D53
:1000700008009F01170A97003C3A031D08009701EA
:10008000220AA2003C3A031D0800A201180A9800A7
:10009000183A031D08009801130A9300073C03183F
:1000A0000800013093000800AE01AF01B101B201B8
:1000B000B001301A08000310B10DB20DA80DA90D42
:1000C000AE0DAF0D2B082F02031D68282A082E0243
:1000D000031C71282A08AE022B08031CAF03AF02D1
:1000E0003114B00A5928031306080317AB002B106C
:1000F000AB102B11AB112B12AB12280E0F39AC0029
:100100000F302C05AA002A182B14AA18AB142A1990
:100110002B15AA19AB15A908031D2B162B080313C1
:1001200086000A300317AC001020031386160A302D
:100130000317AC001020031386120F300317280595
:10014000AA000A30AC001020031306080317AB0006
:100150002B10AB102B11AB112B12AB122A182B1436
:10016000AA18AB142A192B15AA19AB15A908031D37
:100170002B162B08031386000A300317AC0010203F
:10018000031386160A300317AC00102003138612DF
:100190000A300317AC0010200800A41FDC282D3003
:1001A000A8001030A90073202308003CA800A4096F
:1001B0000318A40A2808A3002308A5002408A60001
:1001C00027302402031DE62810302302031C1A29BD
:1001D000A41B1A29AC012508A8002608A900A61FFF
:1001E000F728A809A909A80A0319A90AAC0A103016
:1001F000AA002730AB0054203108A7002C1C02298C
:10020000A709A70A2708303EA8001030A9007320CC
:100210002708003C03181A2910302502A8002730AF
:10022000031C28302602A9002808A5002908A600DA
:10023000A703082903302402031D2029E8302302E4
:10024000031C5529A41B5529AD012508A800260823
:10025000A900A61F3129A809A909A80A0319A90AF2
:10026000AD0AE830AA000330AB0054203108AC00DE
:100270002D1C3C29AC09AC0A2C08A700303EA80074
:100280001030A90073202708003C03185529E830D6
:100290002502A8000330031C04302602A900280808
:1002A000A5002908A600A70343292408803AA8002E
:1002B00080302802031D5E2964302302031C8B2931
:1002C000AD012508A8002608A900A61F6D29A809C8
:1002D000A909A80A0319A90AAD0A6430AA00AB014A
:1002E00054203108AC002D1C7729AC09AC0A2C082D
:1002F000A700303EA8001030A90073202708003C5A
:1003000003188B2964302502A800031CA6032808C3
:10031000A500A7037E292408803AA800803028027F
:10032000031D94290A302302031CC129AD012508AD
:10033000A8002608A900A61FA329A809A909A80A98
:100340000319A90AAD0A0A30AA00AB0154203108EA
:10035000AC002D1CAD29AC09AC0A2C08A700303E1E
:10036000A8001030A90073202708003C0318C129F9
:100370000A302502A800031CA6032808A500A7032D
:10038000B4292508303EA8001030A90073200800C9
:100390002308A8001030A90073200800A408031D3A
:1003A000D4298030A400D629C030A4002308240713
:1003B000A800A90173200230A5001F2008008316A1
:1003C00003139F017F309B00050883120317A300CE
:1003D00083160313060883120317A4001030831634
:1003E000031305048500A13083129F000317A501A4
:1003F000283025020318FE29A50AF8290430031322
:100400001F049F001F19022A0317230883160313D2
:1004100085008312031724088316031386009B01AB
:10042000803083129F000800831203131E080317F5
:10043000A3000800831203171603031D5A2AA30101
:100440000130A400CE210A3014020318332AA3017C
:100450000130A400CE213030A300C8211408A3002D
:10046000A401CD20372A1408A300A401CD20023016
:10047000A3000130A400CE213A30A300C8210330EC
:10048000A3000130A400CE210A301E020318552A11
:100490000330A3000130A400CE213030A300C821D6
:1004A0001E08A300A401CD2008001E08A300A4017B
:1004B000CD2008001808940022089E000130960004
:1004C0000800DF21142223089B001C081B020318CC
:1004D0000800013092000800831203171808073A39
:1004E000031D742A013095001808083A031D7B2A61
:1004F00095019901920118080F3C0318812A0130D7
:1005000095001308043C0318912A1808173A031D94
:10051000982A22083B3A031D982A950199019201D5
:10052000982A1808173A031D982A950199019201F3
:100530001503031DB92A1203031D08000130990099
:10054000F7308316031305058500831203179908F6
:100550000319B42AF730031305050317A300083065
:100560002304031385000800F730031305058500F5
:100570000800F7308316031305058500831203175F
:1005800099080319CD2AF730031305050317A300B3
:1005900008302304031385000800F7300313050512
:1005A00085000800A6012508260203180800831309
:1005B00024188317230826078400800803190800DD
:1005C0008313241883172308260784000008A80033
:1005D0001030A9007320A60AD32A01308312031712
:1005E000A800A90173200230A5001F200230A80036
:1005F000A90173200230A5001F20080061226C228F
:10060000ED220130831603130504850001308312A7
:1006100005050317A300A00123030319A00A200363
:100620000319D32683120317A301A401CE2100309E
:10063000A600DC30A3002608A4001430A500D222B6
:100640000430A300A401CE213D30A300C8210A300C
:1006500018020318372B0530A300A401CE21303037
:10066000A300C8211808A300A401CD203B2B180823
:10067000A300A401CD200730A300A401CE213A306D
:10068000A300C8210A3022020318522B0830A3000D
:10069000A401CE213030A300C8212208A300A40168
:1006A000CD20562B2208A300A401CD200A30A300A0
:1006B000A401CE213A30A300C8210A301702031842
:1006C0006D2B0B30A300A401CE213030A300C82134
:1006D0001708A300A401CD20712B1708A300A401C3
:1006E000CD200E30A300A401CE211303031D822BC5
:1006F0000030A6007530A3002608A4000230A50033
:10070000D222D52B1308023A031D902B0130A600EC
:100710001030A3002608A4000230A500D222D52B59
:100720001308033A031D9E2B0030A6007B30A30064
:100730002608A4000230A500D222D52B1308043AC3
:10074000031DAC2B0030A6007730A3002608A400C0
:100750000230A500D222D52B1308053A031DBA2B6F
:100760000030A6007930A3002608A4000230A500BE
:10077000D222D52B1308063A031DC82B0030A60041
:100780007330A3002608A4000230A500D222D52B86
:100790001308073A031DD52B0030A6007D30A300B7
:1007A0002608A4000230A500D2220730A3000130A1
:1007B000A400CE210030A600A030A3002608A4008B
:1007C0001430A500D2220C30A3000130A400CE21A9
:1007D0003D30A300C8210D30A3000130A400CE217C
:1007E0001B08A300A401CD20A3010130A400CE2149
:1007F0001903031DFD2B1A22022C9601A3010130BF
:10080000A400CE21FF30A5001F20F530A5001F2039
:10081000FE2A83120317C6010330C7001030C80038
:100820006F30C900C908031908004808CA00CB0185
:100830004718CA17C7184B1483134B1883174A0855
:1008400084000008CC007F304C05CD00CC1B532C1D
:10085000CF014D084807CE000318CF0A4E0AD0003A
:10086000490850020318532CD1014718D017C71854
:100870005114831351188317500884000008D200C4
:10088000D21B532C8313511883175008840000087F
:10089000D300530ACC0783134B1883174A088400EC
:1008A0004C088000122CCC134C08C8074908480695
:1008B000031D7E2CC60A46030319672C4608023A1C
:1008C00003196E2C4608033A0319752C7C2C023050
:1008D000C7005430C8006F30C900122C0030C70068
:1008E0000030C8000030C900122C0030C7000030B2
:1008F000C8000030C900122CC901122CC80A122CE1
:10090000831203172003031D962C01308316031353
:10091000050485000130831205050317A300A40117
:1009200023030319A40A2408A000802C83120317B0
:10093000A008031D0800ED22A301A401CE21003070
:10094000A600B430A3002608A4001430A500D222CB
:10095000A3010130A400CE211303031DB92C0030E4
:10096000A6007530A3002608A4000230A500D222FC
:100970000C2D1308023A031DC72C0130A6001030BD
:10098000A3002608A4000230A500D2220C2D1308D3
:10099000033A031DD52C0030A6007B30A3002608A7
:1009A000A4000230A500D2220C2D1308043A031D26
:1009B000E32C0030A6007730A3002608A400023004
:1009C000A500D2220C2D1308053A031DF12C00308E
:1009D000A6007930A3002608A4000230A500D22288
:1009E0000C2D1308063A031DFF2C0030A6007330AF
:1009F000A3002608A4000230A500D2220C2D130863
:100A0000073A031D0C2D0030A6007D30A3002608F8
:100A1000A4000230A500D22202308316031305047D
:100A200085000230831205050317A300A1010230DF
:100A300023020319A10A2103031D392D1308063CC3
:100A4000031C9301130A93002103031D392D023067
:100A5000831603130504850002308312050503176E
:100A6000A300A401023023020319A40A2408A10050
:100A7000242D9630A5001F20013083160313050492
:100A800085000130831205050317A300A401230389
:100A90000319A40A2408A0002003031D962C200398
:100AA000031D632D013083160313050485000130F7
:100AB000831205050317A300A40123030319A40A45
:100AC0002408A0004F2DFE22962CC21F6A2DC401BF
:100AD000C50108004310C6010330C7001030C8002C
:100AE0006F30C900C9080319E52D4808CA00CB01B9
:100AF0004718CA17C7184B1483134B1883174A0893
:100B000084000008CC00CC1BB82D42084C02031C0A
:100B1000B82D80304204CF0083134B1883174A0846
:100B200084004F0880004A08CD004B08CE004C08D6
:100B300042020318B02D420AC8074808CA00CB0178
:100B40004718CA17C7184B1442084C02CF004F036E
:100B5000D00083134B1883174A0884005008800084
:100B6000CD0A0319CE0A4D08C4004E08C50008007E
:100B7000CC134C08C80749084806031DE32DC60AD4
:100B800046030319CC2D4608023A0319D32D460813
:100B9000033A0319DA2DE12D0230C7005430C800A2
:100BA0006F30C900722D0030C7000030C80000301F
:100BB000C900722D0030C7000030C8000030C900E5
:100BC000722DC901722DC80A722D4318EA2D4314E3
:100BD00009246B2DC401C5010800003083120317DE
:100BE000A6002030A3002608A4001430A500D222BD
:100BF000A008031DA42EDF21142223089B0001302E
:100C000083160313050485000130831205050317BD
:100C1000A300A40123030319A40A2408A000A3012C
:100C20000130A400CE2164301C020318232EA3013E
:100C30000130A400CE212030A300C8211C08A3004D
:100C4000A401CD20272E1C08A300A401CD2006302E
:100C5000A3000130A400CE210030A600A030A300E4
:100C60002608A4001430A500D2220B30A3000130C6
:100C7000A400CE213D30A300C82164301B0203181C
:100C80004E2E0C30A3000130A400CE212030A30052
:100C9000C8211B08A300A401CD20522E1B08A300CD
:100CA000A401CD2002308316031305048500023011
:100CB000831205050317A300A101023023020319C3
:100CC000A10A2103031D7B2E1C0A9C002103031D86
:100CD0007B2E023083160313050485000230831235
:100CE00005050317A300A401023023020319A40A77
:100CF0002408A100662E0430831603130504850022
:100D00000430831205050317A3009D01043023025C
:100D100003199D0A1D03031DF82D1C039C001D03D0
:100D2000031DF82D043083160313050485000430D9
:100D3000831205050317A300A4010430230203193D
:100D4000A40A24089D008F2E2003031DB82E013015
:100D5000831603130504850001308312050503176C
:100D6000A300A40123030319A40A2408A000A42EAD
:100D70009901FE30831603130505850083120317BE
:100D800099080319CD2EFE30031305050317A300A0
:100D90000130230403138500D12EFE300313050513
:100DA000850080240800831203172003031DEC2E06
:100DB0009630A5001F20013083160313050485001B
:100DC0000130831205050317A300A40123030319AF
:100DD000A40A2408A000D32EED220030A6005C3027
:100DE000A3002608A4001430A500D222A008031DE9
:100DF0009B2F0230A3000130A400CE210A3018023C
:100E000003180F2F0230A3000130A400CE21303090
:100E1000A300C8211808A300A401CD20132F18088F
:100E2000A300A401CD203A30A300C8210530A300BF
:100E30000130A400CE210A30220203182C2F0530E5
:100E4000A3000130A400CE213030A300C821220825
:100E5000A300A401CD20302F2208A300A401CD209F
:100E60000230831603130504850002308312050542
:100E70000317A300A101023023020319A10A2103D1
:100E8000031D5C2F180A9800183A031998012103D2
:100E9000031D5C2F02308316031305048500023006
:100EA000831205050317A300A401023023020319CE
:100EB000A40A2408A100472F043083160313050455
:100EC00085000430831205050317A3009D0104303B
:100ED000230203199D0A1D03031D8A2F180398007E
:100EE0009808031D752F173098001D03031D8A2FC6
:100EF00004308316031305048500043083120505AE
:100F00000317A300A401043023020319A40A240830
:100F10009D00752F013083160313050485000130F1
:100F2000831205050317A300A40123030319A40AD0
:100F30002408A000F62E2003031DAF2F01308316D6
:100F40000313050485000130831205050317A30070
:100F5000A40123030319A40A2408A0009B2FED2257
:100F60000030A600C830A3002608A4001430A50055
:100F7000D222A0088A15031D67280230A300013081
:100F8000A4008A11CE210A3018020318D42F02308F
:100F9000A3000130A400CE213030A300C8211808DE
:100FA000A300A401CD20D82F1808A300A401CD20B0
:100FB0003A30A300C8210530A3000130A400CE219F
:100FC0000A3022020318F12F0530A3000130A400DB
:100FD000CE213030A300C8212208A300A401CD20D7
:100FE000F52F2208A300A401CD200230831603139D
:100FF000050485000230831205050317A300A40130
:10100000023023020319A40A2408A10021038A152F
:10101000031D2428220AA2003C3A0319A20121033D
:10102000031D2428023083160313050485000230B3
:10103000831205050317A300A4010230230203193C
:10104000A40A2408A1000F28043083160313050402
:1010500085000430831205050317A300A4010430A2
:1010600023020319A40A24089D001D03031D55280B
:101070000130220203183E283B30A2002203A200C6
:101080001D03031D55280430831603130504850032
:101090000430831205050317A300A40104302302C2
:1010A0000319A40A24089D00402801308316031365
:1010B000050485000130831205050317A300A40170
:1010C00023030319A40A2408A0008A11B92F2003BE
:1010D000031D7B28013083160313050485000130AE
:1010E000831205050317A300A40123030319A40A0F
:1010F0002408A00067288A11ED22ED250800BF0111
:101100003D08C2008A1165254408C0004508C10099
:10111000C0088A15031D9328C108031D93283B08A6
:10112000C0003C08C100BE0136083E020318B828C2
:101130003D083F020318B628831324188317230899
:101140003E0784000008C20083134118831740083B
:101150003F07840042088000831324188317230864
:101160003E07840080080319B828BF0ABE0A9428E5
:10117000BE013A083E020318DD283D083F0203186D
:10118000DB2883133818831737083E0784000008CC
:10119000C20083134118831740083F0784004208A8
:1011A000800083133818831737083E0784008008AF
:1011B0000319DD28BF0ABE0AB9283D083F020318FB
:1011C000E92883134118831740083F078400003043
:1011D000800040083B06031DF12841083C06031926
:1011E0000829BE013D083E0203180829831341184F
:1011F000831740083E0784000008C20083133C1890
:1012000083173B083E07840042088000BE0AF2288C
:101210003F08C2000800831603130610861006114B
:101220008611061286120C3083120317A5008A114C
:101230001F203330A800A90173200230A5001F2011
:101240003230A800A90173200230A5001F202C30E5
:10125000A800A90173200230A5001F200630A800B5
:10126000A90173200230A5001F200C30A800A9019D
:1012700073200230A5001F200130A800A9017320AF
:101280000230A5001F200230A800A90173200230FF
:10129000A5001F2008000B21ED222030A900AE0080
:1012A0005330A5006530A700AC006930AF006C304A
:1012B000A8006E30AD00B0007230AB007430A600F4
:1012C0007530AA00B1010130BE002530A3003E08F0
:1012D000A4000C30B600B3010130BE003330B700BB
:1012E0003E08B800BA010030BE005C30BB003E08CA
:1012F000BC001430BD008A157F205430A500693031
:10130000A6006A30A7006430A800A9010130AB0034
:101310002530A3002B08A4000430B600AA01013038
:10132000AB002A30B7002B08B800BA010030AB0080
:10133000DC30BB002B08BC001430BD007F20203007
:10134000A900B1004430AA004730A5006530A600CE
:10135000A700AC00AF006630A8006930B2006C3066
:10136000B0006D30AD006E30B3007030AE00723042
:10137000AB00B4010130BE002530A3003E08A4003C
:101380000F30B600B9010130BE003930B7003E0859
:10139000B800BA010030BE002030BB003E08BC00DF
:1013A0001430BD007F202030A900AD004430A500DE
:1013B0004A30AA004D30AE006130AB006430B0005E
:1013C000B1006530B2006930AF006C30B3006E30F0
:1013D000AC006F30A600A7007230A800B401013045
:1013E000BE002530A3003E08A4000F30B600B901AE
:1013F0000130BE003930B7003E08B800BA010030F5
:10140000BE004830BB003E08BC001430BD007F2049
:101410002030A900AF004430A5006530AA00AD001F
:10142000B2006B30A8006E30AB006F30B10072308C
:10143000A600AE007330B4007430AC00B000B3004E
:101440007530A700B5010130BE002530A3003E086D
:10145000A4001030B600B9010130BE003930B70029
:101460003E08B800BA010030BE003430BB003E0870
:10147000BC001430BD007F204C30A5006930A600B0
:101480006330A7006830A8007430A900AA010130B9
:10149000AC002530A3002C08A4000530B600AB0139
:1014A0000130AC002B30B7002C08B800BA01003076
:1014B000AC00A030BB002C08BC001430BD007F2065
:1014C0002030A900B1005330A5006530A700AF005F
:1014D0006930AB00B2006C30A8006D30AA006E30ED
:1014E000AC00B000B3007430A600AE007530AD00A3
:1014F000B4010130B9002530A3003908A4000F3031
:10150000B600B5010130B9003530B7003908B80070
:10151000BA010030B900C830BB003908BC00143033
:10152000BD007F205A30A5006F30A600A701013012
:10153000A9002530A3002908A4000230B600A801A4
:101540000130A9002830B7002908B800BA010030DE
:10155000A9007D30BB002908BC000230BD007F20FF
:101560004D30A5006130A600A7010130A90025304B
:10157000A3002908A4000230B600A8010130A90088
:101580002830B7002908B800BA010030A90075302A
:10159000BB002908BC000230BD007F204430A500FC
:1015A0006930A600A7010130A9002530A300290851
:1015B000A4000230B600A8010130A9002830B7000D
:1015C0002908B800BA010130A9001030BB00290871
:1015D000BC000230BD007F205730A5006F30A60050
:1015E000A7010130A9002530A3002908A40002307A
:1015F000B600A8010130A9002830B7002908B800BA
:10160000BA010030A9007B30BB002908BC000230C1
:10161000BD007F204430A5006F30A600A701013037
:10162000A9002530A3002908A4000230B600A801B3
:101630000130A9002830B7002908B800BA010030ED
:10164000A9007730BB002908BC000230BD007F2014
:101650005630A5007230A600A7010130A900253040
:10166000A3002908A4000230B600A8010130A90097
:101670002830B7002908B800BA010030A900793035
:10168000BB002908BC000230BD007F205A30A500F5
:101690006130A600A7010130A9002530A300290868
:1016A000A4000230B600A8010130A9002830B7001C
:1016B0002908B800BA010030A9007330BB0029081E
:1016C000BC000230BD007F202030A900AC00B0007B
:1016D0005330A5006130AE006430AA00AD00653023
:1016E000A700AB006730AF006930B1006C30A800D4
:1016F0006E30B2007430A600B3010130B500253061
:10170000A3003508A4000E30B600B4010130B500C6
:101710003430B7003508B800BA010030B500B43035
:10172000BB003508BC001430BD007F200F3098008E
:101730003230A2002D30970064309C0096019A014F
:10174000013093000030A6004830A3002608A40012
:101750001430A5008A11D222A3010130A400CE21A9
:101760000030A6003430A3002608A4001430A500E1
:10177000D222A0088A15031DCE2B01308316031335
:10178000050485000130831205050317A300A40199
:1017900023030319A40A2408A000B92B83160313FA
:1017A00081120116F030010583120317A3000730E0
:1017B00023048316031381008B178B168A11D326FB
:1017C0000800831603139B0107309C00C030810082
:1017D0004B21FE228A15EA2B83120317A301033043
:1017E000A4001030A5006F30A600A6080319080059
:1017F0002608A7002508A7022508A800A901241883
:10180000A817A418291483132918831728088400FB
:1018100027088000A30A23030319172C2308023A80
:1018200003191E2C2308033A0319252C2C2C0230F3
:10183000A4005430A5006F30A600F52B0030A400A2
:101840000030A5000030A600F52B0030A4000030C9
:10185000A5000030A600F52BA601F52B8A150A126B
:10186000EC23E12B0B1D372C8A1132200B11720E49
:101870008400710E8A00700E8300FF0E7F0E090037
:00000001FF
